 mosumac

 Timestamp is 475cde8b (Mon Dec 10 12:06:59 2007)

 Preferred load address is 00010000

 Start         Length     Name                   Class
 0001:00000000 00007d1cH .text                   CODE
 0001:00007d1c 00000284H .text$s                 CODE
 0002:00000000 00000150H .idata$5                DATA
 0002:00000150 000000e8H .rdata                  DATA
 0002:00000238 0000005bH .rdata$debug            DATA
 0002:000002a0 00000008H .rdata$sxdata           DATA
 0002:000002a8 00000034H .xdata$x                DATA
 0003:00000000 00000174H .data                   DATA
 0003:00000174 00000004H .kmdftypeinit$a         DATA
 0003:00000178 00000004H .kmdftypeinit$c         DATA
 0003:00000180 00000bb0H .bss                    DATA
 0004:00000000 00000047H INIT                    CODE
 0004:00000048 00000050H .idata$2                CODE
 0004:00000098 00000014H .idata$3                CODE
 0004:000000ac 00000150H .idata$4                CODE
 0004:000001fc 0000075cH .idata$6                CODE
 0005:00000000 00000058H .rsrc$01                DATA
 0005:00000060 00000388H .rsrc$02                DATA

  Address         Publics by Value              Rva+Base       Lib:Object

 0000:00000002       ___safe_se_handler_count   00000002     <absolute>
 0001:00000006       _MosNdisMiniportHalt@8     00011006 f   mosnhalt.obj
 0001:00000188       _MosNdisMiniportShutdown@8 00011188 f   mosnhalt.obj
 0001:000001da       _MosNdisDevicePnPEventNotifyHandler@8 000111da f   mosnhalt.obj
 0001:000001fa       _MosNdisMiniportCancelSendNetBufferLists@8 000111fa f   mosnhalt.obj
 0001:000002a0       _MosNdisMiniportReset@8    000112a0 f   mosnhalt.obj
 0001:000002f6       _MosNdisMiniportCheckForHang@4 000112f6 f   mosnhalt.obj
 0001:00000320       _MosNdisResetComplete@4    00011320 f   mosnhalt.obj
 0001:00000388       _ResetDispatchThread@4     00011388 f   mosnhalt.obj
 0001:000003fa       _ExAllocateFromNPagedLookasideList@4 000113fa f i mosninit.obj
 0001:0000042c       _ExFreeToNPagedLookasideList@8 0001142c f i mosninit.obj
 0001:0000045e       _MosUsbDeleteDevice@4      0001145e f   mosninit.obj
 0001:00000cde       _MosNdisMiniportSetOptions@8 00011cde f   mosninit.obj
 0001:00000ce8       _MosNdisMiniportInitialize@12 00011ce8 f   mosninit.obj
 0001:000015e6       _MosNdisMiniportPause@8    000125e6 f   mosninit.obj
 0001:00001716       _MosNdisMiniportRestart@8  00012716 f   mosninit.obj
 0001:000017c4       _TerminateThreads@4        000127c4 f   mosninit.obj
 0001:00001812       _FreeResourceAllocation@4  00012812 f   mosninit.obj
 0001:000018f8       _MosNdisCompleteOidRequestMediaStatus@4 000128f8 f   mosninit.obj
 0001:00001998       _MosNdisIndicateConnectionStatus@8 00012998 f   mosninit.obj
 0001:00001ab8       _MosNdisMiniportUnload@4   00012ab8 f   mosninit.obj
 0001:00001ae0       _DriverEntry@8             00012ae0 f   mosninit.obj
 0001:00001bf2       _MP_RECEIVE_STATS@8        00012bf2 f i mosnrecv.obj
 0001:00001cfa       _MosNdisIndicateRxPacketToNdis@4 00012cfa f   mosnrecv.obj
 0001:00002256       _MosUsbSetupRead@12        00013256 f   mosnrecv.obj
 0001:00002336       _MosUsbCancelPendingRxIrpsWDM@4 00013336 f   mosnrecv.obj
 0001:000023ac       _LoopBackSetupRead@12      000133ac f   mosnrecv.obj
 0001:00002532       _CancelRxPendingIRPs@4     00013532 f   mosnrecv.obj
 0001:00002658       _MosNdisMiniportReturnNetBufferLists@12 00013658 f   mosnrecv.obj
 0001:00002760       _SetupNextRxPacket@8       00013760 f   mosnrecv.obj
 0001:00002a3a       _PhyStatusRegDispatchThread@4 00013a3a f   mosnrecv.obj
 0001:00002a92       _RxThreadedDpc@16          00013a92 f   mosnrecv.obj
 0001:00002aaa       _ParseRegistryParameters@8 00013aaa f   mosnregparam.obj
 0001:00002eb8       _MPFillPoMgmtCaps@16       00013eb8 f   mosnrequest.obj
 0001:00002ee8       _MPSetPower@8              00013ee8 f   mosnrequest.obj
 0001:00002f58       _MosNdisMiniportCancelOidRequest@8 00013f58 f   mosnrequest.obj
 0001:00002fc4       _MosNdisMiniportSetInformation@8 00013fc4 f   mosnrequest.obj
 0001:00003254       _RequestDispatchThread@4   00014254 f   mosnrequest.obj
 0001:000032a4       _PowerDispatchThread@4     000142a4 f   mosnrequest.obj
 0001:000032f6       _MosNdisGetStatsCounters@12 000142f6 f   mosnrequest.obj
 0001:00003642       _MosNdisMiniportQueryInformation@8 00014642 f   mosnrequest.obj
 0001:00004ddc       _MosNdisMiniportOidRequest@8 00015ddc f   mosnrequest.obj
 0001:00004e1a       _MP_FREE_SEND_NET_BUFFER@8 00015e1a f i mosnsend.obj
 0001:00004e46       _MosNdisInsertTcbToQueue@4 00015e46 f   mosnsend.obj
 0001:00004f54       _MosUsbCancelPendingTxIrps@4 00015f54 f   mosnsend.obj
 0001:00004f86       _LoopBackSetupWrite@12     00015f86 f   mosnsend.obj
 0001:0000509e       _MP_SEND_STATS@8           0001609e f i mosnsend.obj
 0001:000051b4       _CancelTxPendingIRPs@4     000161b4 f   mosnsend.obj
 0001:000053c0       _CancelTxPendingPackets@4  000163c0 f   mosnsend.obj
 0001:00005526       _CompleteSendNetBufferListsWithError@20 00016526 f   mosnsend.obj
 0001:00005560       _MpCopyNetBuffer@12        00016560 f   mosnsend.obj
 0001:000056b2       _MiniportSendNetBufferList@16 000166b2 f   mosnsend.obj
 0001:000057fe       _MosNdisMiniportSendNetBufferLists@16 000167fe f   mosnsend.obj
 0001:00005984       _MosNdisMoveTCBFromUSBPendingToNdisPendingListHead@8 00016984 f   mosnsend.obj
 0001:00005c02       _MosUsbSetupWrite@16       00016c02 f   mosnsend.obj
 0001:00005d50       _SetupTxDequeuePacket@4    00016d50 f   mosnsend.obj
 0001:00005f1e       _TxThreadedDpc@16          00016f1e f   mosnsend.obj
 0001:00005f1e       _ScheduleTxPacket@16       00016f1e f   mosnsend.obj
 0001:0000617c       _MosUsbSaveMulticastList@20 0001717c f   mosuinit.obj
 0001:0000622e       _UpdateHifReg15@8          0001722e f   mosuinit.obj
 0001:00006260       _SetLinkValues@8           00017260 f i mosuinit.obj
 0001:000062fe       _MosUsbReadPhyStatusReg@4  000172fe f   mosuinit.obj
 0001:0000658a       _MosUsbEPROMWrite@12       0001758a f   mosuinit.obj
 0001:000066bc       _MosUsbWriteMacToHIF@12    000176bc f   mosuinit.obj
 0001:0000672a       _MosUsbEPROMDataWrite@12   0001772a f   mosuinit.obj
 0001:000067f2       _MosUsbEPROMRead@12        000177f2 f   mosuinit.obj
 0001:00006814       _MosUsbGetCurrentConnectionStatus@8 00017814 f   mosuinit.obj
 0001:0000684c       _MosUsbReadStringDescriptor@12 0001784c f   mosuinit.obj
 0001:00006916       _MosUsbStartDevice@4       00017916 f   mosuinit.obj
 0001:00006f84       _MosUsbSetPacketFilter@4   00017f84 f   mosuinit.obj
 0001:00007022       _CardFillMulticastRegs@12  00018022 f   mosumulti.obj
 0001:000070a8       _SetVendorCommandPassive@24 000180a8 f   mosuvendor.obj
 0001:0000715c       _GetVendorCommandPassive@24 0001815c f   mosuvendor.obj
 0001:0000720c       _ReadPhyRegisterPassive@12 0001820c f   mosuvendor.obj
 0001:000072ca       _WritePhyRegisterPassive@12 000182ca f   mosuvendor.obj
 0001:00007354       _SetResetLoopBack@12       00018354 f   mosuvendor.obj
 0001:0000740c       _Get_SetVendorCommand@28   0001840c f   mosuvendor.obj
 0001:00007442       _ResetPortFreeSyncObjs@4   00018442 f   mosureset.obj
 0001:00007480       _ResetPort@4               00018480 f   mosureset.obj
 0001:000074f6       _MosUsbResetBulkOut@4      000184f6 f   mosureset.obj
 0001:00007524       _MosUsbResetBulkIn@4       00018524 f   mosureset.obj
 0001:00007552       _ReInitializeDevice@4      00018552 f   mosureset.obj
 0001:000075c8       _ResetPortDispatchThread@4 000185c8 f   mosureset.obj
 0001:00007622       _CallBack_ResetEndPoint@8  00018622 f   mosureset.obj
 0001:000076f2       _MosUsbSetPower@4          000186f2 f   mosuidle.obj
 0001:0000774c       @__security_check_cookie@4 0001874c f   BufferOverflowK:secchk.obj
 0001:00007760       ___report_gsfailure        00018760 f   BufferOverflowK:gs_report.obj
 0001:0000778c       _KeGetCurrentThread@0      0001878c f   ntoskrnl:ntoskrnl.exe
 0001:00007798       _memset                    00018798 f   ntoskrnl:ntoskrnl.exe
 0001:000077a4       _DbgPrint                  000187a4 f   ntoskrnl:ntoskrnl.exe
 0001:000077b0       __allmul                   000187b0 f   ntoskrnl:ntoskrnl.exe
 0001:000077bc       _memcpy                    000187bc f   ntoskrnl:ntoskrnl.exe
 0001:000077c8       __SEH_prolog4_GS           000187c8 f   ntoskrnl:sehprolg4gs.obj
 0001:00007810       __SEH_epilog4_GS           00018810 f   ntoskrnl:sehprolg4gs.obj
 0001:00007830       __except_handler4          00018830 f   ntoskrnl:chandler4.obj
 0001:0000798c       __SEH_prolog4              0001898c f   ntoskrnl:sehprolg4.obj
 0001:000079d1       __SEH_epilog4              000189d1 f   ntoskrnl:sehprolg4.obj
 0001:000079ec       __local_unwind4            000189ec f   ntoskrnl:exsup4.obj
 0001:00007ac2       __seh_longjmp_unwind4@4    00018ac2 f   ntoskrnl:exsup4.obj
 0001:00007ade       @_EH4_CallFilterFunc@8     00018ade f   ntoskrnl:exsup4.obj
 0001:00007af5       @_EH4_TransferToHandler@8  00018af5 f   ntoskrnl:exsup4.obj
 0001:00007b0e       @_EH4_GlobalUnwind@4       00018b0e f   ntoskrnl:exsup4.obj
 0001:00007b28       @_EH4_LocalUnwind@16       00018b28 f   ntoskrnl:exsup4.obj
 0001:00007b44       __NLG_Notify1              00018b44 f   ntoskrnl:_nlgsupp.obj
 0001:00007b4d       __NLG_Notify               00018b4d f   ntoskrnl:_nlgsupp.obj
 0001:00007b64       __NLG_Dispatch2            00018b64     ntoskrnl:_nlgsupp.obj
 0001:00007b64       __NLG_Dispatch             00018b64     ntoskrnl:_nlgsupp.obj
 0001:00007b6c       __NLG_Call                 00018b6c f   ntoskrnl:_nlgsupp.obj
 0001:00007b6e       __NLG_Return2              00018b6e     ntoskrnl:_nlgsupp.obj
 0001:00007b74       _RtlUnwind@16              00018b74 f   ntoskrnl:ntoskrnl.exe
 0001:00007b7f       ?FxStubDriverUnloadCommon@@YGXXZ 00018b7f f   WdfDriverEntry:stub.obj
 0001:00007bb5       _FxStubDriverUnload@4      00018bb5 f   WdfDriverEntry:stub.obj
 0001:00007bdd       _FxStubDriverMiniportUnload@8 00018bdd f   WdfDriverEntry:stub.obj
 0001:00007bea       _FxDriverEntry@8           00018bea f   WdfDriverEntry:stub.obj
 0001:00007ccd       ?FxStubInitTypes@@YGXXZ    00018ccd f   WdfDriverEntry:inittypes.obj
 0001:00007d0a       _WdfVersionUnbind@12       00018d0a f   WdfLdr:WDFLDR.SYS
 0001:00007d16       _WdfVersionBind@16         00018d16 f   WdfLdr:WDFLDR.SYS
 0001:00007d1c       ??_C@_0DC@JGKDAAMJ@NdisWriteConfiguration?$CI?$CJ?5for?5MAC@FNODOBFM@ 00018d1c     mosninit.obj
 0001:00007d4e       ??_C@_0DG@KCINMJDM@NdisWriteConfiguration?$CI?$CJ?5for?5MAC@FNODOBFM@ 00018d4e     mosninit.obj
 0001:00007d84       ??_C@_0CB@FBBMJBPN@?5StringData?4MaximumLength?5?$DN?5?$CFd?5?6@FNODOBFM@ 00018d84     mosninit.obj
 0001:00007da6       ??_C@_0BK@GHNHCLCL@?5StringData?4Length?5?$DN?5?$CFd?5?6?$AA@FNODOBFM@ 00018da6     mosninit.obj
 0001:00007dc0       ??_C@_0CJ@BNGLENBL@Trying?5to?5make?5the?5NetworkAddres@FNODOBFM@ 00018dc0     mosninit.obj
 0001:00007dea       ??_C@_13COJANIEC@?$AA0?$AA?$AA@FNODOBFM@ 00018dea     mosninit.obj
 0001:00007dee       ??_C@_13JGCMLPCH@?$AA1?$AA?$AA@FNODOBFM@ 00018dee     mosninit.obj
 0001:00007df2       ??_C@_1BO@HGPPFMIN@?$AAN?$AAe?$AAt?$AAw?$AAo?$AAr?$AAk?$AAA?$AAd?$AAd?$AAr?$AAe?$AAs?$AAs?$AA?$AA@FNODOBFM@ 00018df2     mosninit.obj
 0001:00007e10       ??_C@_19HBDGONDF@?$AAI?$AAP?$AAG?$AA1?$AA?$AA@FNODOBFM@ 00018e10     mosnregparam.obj
 0001:00007e1a       ??_C@_17KGECJBCD@?$AAI?$AAP?$AAG?$AA?$AA@FNODOBFM@ 00018e1a     mosnregparam.obj
 0001:00007e22       ??_C@_1CC@KAGCFGJ@?$AAI?$AAP?$AAG?$AAI?$AAP?$AAG?$AA1?$AA_?$AAF?$AAo?$AAr?$AA_?$AAM?$AAo?$AAd?$AAe?$AA?$AA@FNODOBFM@ 00018e22     mosnregparam.obj
 0001:00007e44       ??_C@_1BI@OGHLFKPH@?$AAR?$AAx?$AAT?$AAh?$AAr?$AAe?$AAs?$AAh?$AAo?$AAl?$AAd?$AA?$AA@FNODOBFM@ 00018e44     mosnregparam.obj
 0001:00007e5c       ??_C@_1BI@FGEGAIKH@?$AAT?$AAx?$AAT?$AAh?$AAr?$AAe?$AAs?$AAh?$AAo?$AAl?$AAd?$AA?$AA@FNODOBFM@ 00018e5c     mosnregparam.obj
 0001:00007e74       ??_C@_1CC@GAPLEEKP@?$AAM?$AAu?$AAl?$AAt?$AAi?$AAp?$AAl?$AAe?$AAI?$AAr?$AAp?$AAI?$AAn?$AA2?$AA_?$AA0?$AA?$AA@FNODOBFM@ 00018e74     mosnregparam.obj
 0001:00007e96       ??_C@_19JNKOAPNJ@?$AAR?$AAC?$AAB?$AAS?$AA?$AA@FNODOBFM@ 00018e96     mosnregparam.obj
 0001:00007ea0       ??_C@_19JALAHPJO@?$AAT?$AAC?$AAB?$AAS?$AA?$AA@FNODOBFM@ 00018ea0     mosnregparam.obj
 0001:00007eaa       ??_C@_1CI@EFPCMLOP@?$AAT?$AAh?$AAr?$AAe?$AAs?$AAh?$AAo?$AAl?$AAd?$AAD?$AAi?$AAf?$AAf?$AAe?$AAr?$AAe?$AAn?$AAc?$AAe?$AA?$AA@FNODOBFM@ 00018eaa     mosnregparam.obj
 0001:00007ed2       ??_C@_1BI@PBLMBPJM@?$AAP?$AAa?$AAu?$AAs?$AAe?$AAF?$AAr?$AAa?$AAm?$AAe?$AAs?$AA?$AA@FNODOBFM@ 00018ed2     mosnregparam.obj
 0001:00007eea       ??_C@_1DA@LFGMFGBL@?$AAS?$AAe?$AAt?$AAP?$AAo?$AAw?$AAe?$AAr?$AAD?$AAe?$AAl?$AAa?$AAy?$AAI?$AAn?$AAM?$AAi?$AAl?$AAl?$AAi?$AAS?$AAe?$AAc?$AA?$AA@FNODOBFM@ 00018eea     mosnregparam.obj
 0001:00007f1a       ??_C@_19OLACBGCE@?$AAF?$AAP?$AAG?$AAA?$AA?$AA@FNODOBFM@ 00018f1a     mosnregparam.obj
 0001:00007f24       ??_C@_1BO@HPPMMBKL@?$AAP?$AAa?$AAu?$AAs?$AAe?$AAT?$AAh?$AAr?$AAe?$AAs?$AAh?$AAo?$AAl?$AAd?$AA?$AA@FNODOBFM@ 00018f24     mosnregparam.obj
 0001:00007f42       ??_C@_1BE@GJIEHEGO@?$AAP?$AAa?$AAu?$AAs?$AAe?$AAT?$AAi?$AAm?$AAe?$AA?$AA@FNODOBFM@ 00018f42     mosnregparam.obj
 0001:00007f56       ??_C@_1BG@KFFANNMM@?$AAD?$AAu?$AAp?$AAl?$AAe?$AAx?$AAM?$AAo?$AAd?$AAe?$AA?$AA@FNODOBFM@ 00018f56     mosnregparam.obj
 0001:00007f6c       ??_C@_0DE@GIDKFGMF@NDIS?9WDM?5Driver?5for?5HighSpeed?5US@FNODOBFM@ 00018f6c     mosnrequest.obj
 0002:00000000       __imp__KeGetCurrentIrql@0  00019000     hal:HAL.dll
 0002:00000004       __imp_@KfReleaseSpinLock@8 00019004     hal:HAL.dll
 0002:00000008       __imp_@KfAcquireSpinLock@4 00019008     hal:HAL.dll
 0002:0000000c       \177HAL_NULL_THUNK_DATA    0001900c     hal:HAL.dll
 0002:00000010       __imp__NdisAllocateIoWorkItem@4 00019010     ndis:NDIS.SYS
 0002:00000014       __imp__NdisQueueIoWorkItem@12 00019014     ndis:NDIS.SYS
 0002:00000018       __imp__NdisReadConfiguration@20 00019018     ndis:NDIS.SYS
 0002:0000001c       __imp__NdisMPauseComplete@4 0001901c     ndis:NDIS.SYS
 0002:00000020       __imp__NdisMIndicateReceiveNetBufferLists@20 00019020     ndis:NDIS.SYS
 0002:00000024       __imp__NdisMRegisterMiniportDriver@20 00019024     ndis:NDIS.SYS
 0002:00000028       __imp__NdisMDeregisterMiniportDriver@4 00019028     ndis:NDIS.SYS
 0002:0000002c       __imp__NdisMIndicateStatusEx@8 0001902c     ndis:NDIS.SYS
 0002:00000030       __imp__NdisMOidRequestComplete@12 00019030     ndis:NDIS.SYS
 0002:00000034       __imp__NdisMGetDeviceProperty@24 00019034     ndis:NDIS.SYS
 0002:00000038       __imp__NdisMSetMiniportAttributes@8 00019038     ndis:NDIS.SYS
 0002:0000003c       __imp__NdisOpenConfigurationEx@8 0001903c     ndis:NDIS.SYS
 0002:00000040       __imp__NdisFreeIoWorkItem@4 00019040     ndis:NDIS.SYS
 0002:00000044       __imp__NdisWriteConfiguration@16 00019044     ndis:NDIS.SYS
 0002:00000048       __imp__NdisInitializeTimer@12 00019048     ndis:NDIS.SYS
 0002:0000004c       __imp__NdisCloseConfiguration@4 0001904c     ndis:NDIS.SYS
 0002:00000050       __imp__NdisFreeNetBufferList@4 00019050     ndis:NDIS.SYS
 0002:00000054       __imp__NdisFreeNetBufferListPool@4 00019054     ndis:NDIS.SYS
 0002:00000058       __imp__NdisAllocateNetBufferListPool@8 00019058     ndis:NDIS.SYS
 0002:0000005c       __imp__NdisAllocateMdl@12  0001905c     ndis:NDIS.SYS
 0002:00000060       __imp__NdisAllocateNetBufferAndNetBufferList@24 00019060     ndis:NDIS.SYS
 0002:00000064       __imp__NdisFreeMdl@4       00019064     ndis:NDIS.SYS
 0002:00000068       __imp__NdisAllocateMemoryWithTagPriority@16 00019068     ndis:NDIS.SYS
 0002:0000006c       __imp__NdisFreeMemory@12   0001906c     ndis:NDIS.SYS
 0002:00000070       __imp__NdisMResetComplete@12 00019070     ndis:NDIS.SYS
 0002:00000074       __imp__NdisMSendNetBufferListsComplete@12 00019074     ndis:NDIS.SYS
 0002:00000078       __imp__NdisMSleep@4        00019078     ndis:NDIS.SYS
 0002:0000007c       __imp__NdisReadNetworkAddress@16 0001907c     ndis:NDIS.SYS
 0002:00000080       \177NDIS_NULL_THUNK_DATA   00019080     ndis:NDIS.SYS
 0002:00000084       __imp__WdfVersionUnbind@12 00019084     WdfLdr:WDFLDR.SYS
 0002:00000088       __imp__WdfVersionBind@16   00019088     WdfLdr:WDFLDR.SYS
 0002:0000008c       \177WDFLDR_NULL_THUNK_DATA 0001908c     WdfLdr:WDFLDR.SYS
 0002:00000090       __imp__KeInsertQueueDpc@12 00019090     ntoskrnl:ntoskrnl.exe
 0002:00000094       __imp__IoFreeIrp@4         00019094     ntoskrnl:ntoskrnl.exe
 0002:00000098       __imp_@IofCallDriver@8     00019098     ntoskrnl:ntoskrnl.exe
 0002:0000009c       __imp__IoAllocateIrp@8     0001909c     ntoskrnl:ntoskrnl.exe
 0002:000000a0       __imp__IoReleaseCancelSpinLock@4 000190a0     ntoskrnl:ntoskrnl.exe
 0002:000000a4       __imp__IoCancelIrp@4       000190a4     ntoskrnl:ntoskrnl.exe
 0002:000000a8       __imp__MmUnlockPages@4     000190a8     ntoskrnl:ntoskrnl.exe
 0002:000000ac       __imp__IoFreeMdl@4         000190ac     ntoskrnl:ntoskrnl.exe
 0002:000000b0       __imp__memcpy              000190b0     ntoskrnl:ntoskrnl.exe
 0002:000000b4       __imp__IoAllocateMdl@20    000190b4     ntoskrnl:ntoskrnl.exe
 0002:000000b8       __imp__RtlCompareMemory@12 000190b8     ntoskrnl:ntoskrnl.exe
 0002:000000bc       __imp__IoBuildDeviceIoControlRequest@36 000190bc     ntoskrnl:ntoskrnl.exe
 0002:000000c0       __imp__KeTickCount         000190c0     ntoskrnl:ntoskrnl.exe
 0002:000000c0       _KeTickCount               000190c0     ntoskrnl:ntoskrnl.exe
 0002:000000c4       __imp__KeBugCheckEx@20     000190c4     ntoskrnl:ntoskrnl.exe
 0002:000000c8       __imp__RtlUnwind@16        000190c8     ntoskrnl:ntoskrnl.exe
 0002:000000cc       __imp_@KefAcquireSpinLockAtDpcLevel@4 000190cc     ntoskrnl:ntoskrnl.exe
 0002:000000d0       __imp_@KefReleaseSpinLockFromDpcLevel@4 000190d0     ntoskrnl:ntoskrnl.exe
 0002:000000d4       __imp__MmMapLockedPagesSpecifyCache@24 000190d4     ntoskrnl:ntoskrnl.exe
 0002:000000d8       __imp___allmul             000190d8     ntoskrnl:ntoskrnl.exe
 0002:000000dc       __imp__ExAllocatePoolWithTag@12 000190dc     ntoskrnl:ntoskrnl.exe
 0002:000000e0       __imp__ExFreePoolWithTag@8 000190e0     ntoskrnl:ntoskrnl.exe
 0002:000000e4       __imp__RtlInitUnicodeString@8 000190e4     ntoskrnl:ntoskrnl.exe
 0002:000000e8       __imp__DbgPrint            000190e8     ntoskrnl:ntoskrnl.exe
 0002:000000ec       __imp__KeQueryActiveProcessorCount@4 000190ec     ntoskrnl:ntoskrnl.exe
 0002:000000f0       __imp__KeInitializeThreadedDpc@12 000190f0     ntoskrnl:ntoskrnl.exe
 0002:000000f4       __imp__KeSetTargetProcessorDpc@8 000190f4     ntoskrnl:ntoskrnl.exe
 0002:000000f8       __imp__KeInitializeEvent@12 000190f8     ntoskrnl:ntoskrnl.exe
 0002:000000fc       __imp__PsCreateSystemThread@28 000190fc     ntoskrnl:ntoskrnl.exe
 0002:00000100       __imp__ObReferenceObjectByHandle@24 00019100     ntoskrnl:ntoskrnl.exe
 0002:00000104       __imp__ZwClose@4           00019104     ntoskrnl:ntoskrnl.exe
 0002:00000108       __imp_@ExfInterlockedRemoveHeadList@8 00019108     ntoskrnl:ntoskrnl.exe
 0002:0000010c       __imp__ExDeleteNPagedLookasideList@4 0001910c     ntoskrnl:ntoskrnl.exe
 0002:00000110       __imp__ExInitializeNPagedLookasideList@28 00019110     ntoskrnl:ntoskrnl.exe
 0002:00000114       __imp__memset              00019114     ntoskrnl:ntoskrnl.exe
 0002:00000118       __imp_@ExfInterlockedInsertTailList@12 00019118     ntoskrnl:ntoskrnl.exe
 0002:0000011c       __imp_@InterlockedPushEntrySList@8 0001911c     ntoskrnl:ntoskrnl.exe
 0002:00000120       __imp_@InterlockedPopEntrySList@4 00019120     ntoskrnl:ntoskrnl.exe
 0002:00000124       __imp__KeGetCurrentThread@0 00019124     ntoskrnl:ntoskrnl.exe
 0002:00000128       __imp__KeSetPriorityThread@8 00019128     ntoskrnl:ntoskrnl.exe
 0002:0000012c       __imp__PsTerminateSystemThread@4 0001912c     ntoskrnl:ntoskrnl.exe
 0002:00000130       __imp__KeSetEvent@12       00019130     ntoskrnl:ntoskrnl.exe
 0002:00000134       __imp__KeWaitForSingleObject@20 00019134     ntoskrnl:ntoskrnl.exe
 0002:00000138       __imp__KeClearEvent@4      00019138     ntoskrnl:ntoskrnl.exe
 0002:0000013c       __imp__RtlCopyUnicodeString@8 0001913c     ntoskrnl:ntoskrnl.exe
 0002:00000140       __imp__KeRemoveQueueDpc@4  00019140     ntoskrnl:ntoskrnl.exe
 0002:00000144       __imp__MmProbeAndLockPages@12 00019144     ntoskrnl:ntoskrnl.exe
 0002:00000148       __imp__KeDelayExecutionThread@12 00019148     ntoskrnl:ntoskrnl.exe
 0002:0000014c       \177ntoskrnl_NULL_THUNK_DATA 0001914c     ntoskrnl:ntoskrnl.exe
 0002:0000016c       ??_C@_0BA@MCIECMKL@WDF_DEVICE_INFO?$AA@ 0001916c     mosnhalt.obj
 0002:000001d8       ??_C@_1BI@BJCKEEDJ@?$AAK?$AAm?$AAd?$AAf?$AAL?$AAi?$AAb?$AAr?$AAa?$AAr?$AAy?$AA?$AA@ 000191d8     WdfDriverEntry:stub.obj
 0002:000001f0       __load_config_used         000191f0     ntoskrnl:loadcfg.obj
 0002:000002a0       ___safe_se_handler_table   000192a0     <linker-defined>
 0003:00000000       __WDF_WDF_DEVICE_INFO_TYPE_INFO 0001a000     mosnhalt.obj
 0003:00000018       _SupportedOids             0001a018     mosninit.obj
 0003:00000138       _GlobalResetPortSuccess    0001a138     mosnrequest.obj
 0003:0000013c       ___security_cookie         0001a13c     BufferOverflowK:gs_support.obj
 0003:00000140       ___security_cookie_complement 0001a140     BufferOverflowK:gs_support.obj
 0003:00000144       __NLG_Destination          0001a144     ntoskrnl:_nlgsupp.obj
 0003:00000174       ?__KMDF_TYPE_INIT_START@@3PAPAXA 0001a174     WdfDriverEntry:inittypes.obj
 0003:00000178       ?__KMDF_TYPE_INIT_END@@3PAPAXA 0001a178     WdfDriverEntry:inittypes.obj
 0003:00000180       _gDebugEnable              0001a180     mosnhalt.obj
 0003:00000188       _gbEepromProgrmming        0001a188     mosninit.obj
 0003:00000189       _gbNdisContextAddedToGlobalList 0001a189     mosninit.obj
 0003:0000018a       _GlobalDeviceCountChanged  0001a18a     mosninit.obj
 0003:0000018c       _NdisDeviceHandle          0001a18c     mosninit.obj
 0003:00000190       _DriverInstanceCount       0001a190     mosninit.obj
 0003:00000194       _MiniportDriverContext     0001a194     mosninit.obj
 0003:00000198       _NdisMiniportDriverHandle  0001a198     mosninit.obj
 0003:000001b0       _WdfFunctions              0001a1b0     WdfDriverEntry:stub.obj
 0003:000007bc       _typeWDF_IFR_HEADER        0001a7bc     WdfDriverEntry:stub.obj
 0003:000007d0       _WdfDriverGlobals          0001a7d0     WdfDriverEntry:stub.obj
 0003:000009e0       _WdfClassExtensionList     0001a9e0     WdfDriverEntry:stub.obj
 0003:000009e4       _gbSetPowerDelay           0001a9e4     <common>
 0003:00000a00       _GlobalMosNdisContext      0001aa00     <common>
 0003:00000d20       _DriverVersion             0001ad20     <common>
 0003:00000d28       _GlobalNdisSpinLock        0001ad28     <common>
 0004:00000005       _GsDriverEntry@8           0001b005 f   BufferOverflowK:gs_support.obj
 0004:00000048       __IMPORT_DESCRIPTOR_ntoskrnl 0001b048     ntoskrnl:ntoskrnl.exe
 0004:0000005c       __IMPORT_DESCRIPTOR_HAL    0001b05c     hal:HAL.dll
 0004:00000070       __IMPORT_DESCRIPTOR_NDIS   0001b070     ndis:NDIS.SYS
 0004:00000084       __IMPORT_DESCRIPTOR_WDFLDR 0001b084     WdfLdr:WDFLDR.SYS
 0004:00000098       __NULL_IMPORT_DESCRIPTOR   0001b098     ntoskrnl:ntoskrnl.exe

 entry point at        0001:00007bea

 Static symbols

 0001:000004ca       _FreePhyStatusRegThreadAllocation@4 000114ca f   mosninit.obj
 0001:000004fe       _FreeRequestThreadAllocation@4 000114fe f   mosninit.obj
 0001:00000532       _FreeResetThreadAllocation@4 00011532 f   mosninit.obj
 0001:00000566       _SetupTransmitQueues@4     00011566 f   mosninit.obj
 0001:00000800       _SetupReceiveQueues@4      00011800 f   mosninit.obj
 0001:000009ce       _FreeReceiveAndTransmitQueues@4 000119ce f   mosninit.obj
 0001:00000b0a       _FreeAdapterObject@4       00011b0a f   mosninit.obj
 0001:00000b26       _ResetSynchObjAlloc@4      00011b26 f   mosninit.obj
 0001:00000b94       _RequestSynchObjAlloc@4    00011b94 f   mosninit.obj
 0001:00000c02       _PowerSynchObjAlloc@4      00011c02 f   mosninit.obj
 0001:00000c70       _PhyStatusRegSynchObjAlloc@4 00011c70 f   mosninit.obj
 0001:00001c98       _MoveRcbToFreeList@12      00012c98 f   mosnrecv.obj
 0001:00001fee       _ReadComplete@12           00012fee f   mosnrecv.obj
 0001:0000249c       _GetRcbFromUsbPendingListAndSetCancelFlag@4 0001349c f   mosnrecv.obj
 0001:000024ea       _MoveRcbFromUsbPendingToFreeList@8 000134ea f   mosnrecv.obj
 0001:00002984       _ReadPhyStatusReg@4        00013984 f   mosnrecv.obj
 0001:0000313c       _SetupRequest@4            0001413c f   mosnrequest.obj
 0001:000031da       _PowerRequest@4            000141da f   mosnrequest.obj
 0001:00005146       _PopTcbFromNdisPendingList@8 00016146 f   mosnsend.obj
 0001:00005182       _PushTcbToFreeList@8       00016182 f   mosnsend.obj
 0001:000059d2       _WriteComplete@16          000169d2 f   mosnsend.obj
 0001:00005f46       _SelectInterfaces@4        00016f46 f   mosuinit.obj
 0001:00006062       _ConfigureDevice@4         00017062 f   mosuinit.obj
 0001:00006114       _ResetPortAllocSyncObjs@4  00017114 f   mosuinit.obj
 0001:00007a7c       __unwind_handler4          00018a7c f   ntoskrnl:exsup4.obj
